:1000000010C017C016C015C014C013C012C011C054
:1000100010C00FC00EC00DC00CC00BC00AC009C07C
:1000200008C011241FBECFE5D1E0DEBFCDBF02D096
:1000300044C0E6CF1ABA17BA80E88ABB8BBB2FE759
:1000400034E84EE1215030404040E1F700C000006C
:100050001BBA9FE724E83EE1915020403040E1F791
:1000600000C000008BBB4FE794E82EE14150904068
:100070002040E1F700C000001BBA3FE744E89EE1E2
:10008000315040409040E1F700C000008BBB2FE7AB
:1000900034E84EE1215030404040E1F700C000001C
:1000A0001BBA9FE720EF3AEF42E0915020403040EA
:0E00B0004040D9F700C00000C1CFF894FFCF48
:00000001FF
